:020000040000FA
:0C0000000000000009EF04F023EF04F002
:0800180062EF04F09EA8FED780
:10002000AD6E12000E6A0D6EFF0E0D260E2200D070
:10003000D8A01200030E0A6EE60E02D8F5D70A6A9F
:10004000FE0F096EE86A0A5AD8A0120000000906DD
:1000500000D0F8D70A6A096E110EFF0F09360A366A
:10006000FCE3096E1200E65005E1206A216A226A6B
:10007000236A1200206EE6CF21F0E6CF22F0E6CF11
:1000800023F021BE219E13D823C027F022C026F0E2
:1000900021C025F020C024F014C023F013C022F0AA
:1000A00012C021F011C020F027EC03F021D121BEB5
:1000B00009D12052D8B406D12AC015F02A8C7E0E60
:1000C000205C166E7E0E206E276A266A256A7F0ED9
:1000D000246EF30E235C040ED8A0050E225C350EB0
:1000E000D8A0360E215C02E3BCD903D0202AB9D9AE
:1000F000160623C009F022C00AF021C00BF020C070
:100100000CF0710E276E5F0E266E550E256E800E5A
:10011000246EA9D909C027F00AC026F00BC025F02B
:100120000CC024F027EC03F0C60E276EF50E266EE9
:100130001F0E256E800E246E96D923C00DF022C0AE
:100140000EF021C00FF020C010F009C023F00AC04B
:1001500022F00BC021F00CC020F08A0E276E120E88
:10016000266E790E256E7D0E246E27EC03F0F60EBA
:10017000276E460E266E550E256E7E0E246E73D9A2
:100180000DC027F00EC026F00FC025F010C024F0DF
:10019000F8D923C00DF022C00EF021C00FF020C00E
:1001A00010F00C50206E246E0B50216E256E0A50FC
:1001B000226E266E0950236E276E27EC03F023C0B3
:1001C00018F022C019F021C01AF020C01BF00DC099
:1001D00027F00EC026F00FC025F010C024F027EC49
:1001E00003F009C027F00AC026F00BC025F00CC0B0
:1001F00024F027EC03F018C027F019C026F01AC02D
:1002000025F01BC024F0246624062BD909C027F052
:100210000AC026F00BC025F00CC024F024D91652D9
:1002200052E023C018F022C019F021C01AF020C0FB
:100230001BF016C020F0000E20BEFF0E216E226EB5
:10024000236ECEEC03F023C009F022C00AF021C0D7
:100250000BF020C00CF0830E276E800E266EDE0E93
:10026000256E720E246EF3D918C027F019C026F03F
:100270001AC025F01BC024F0F6D823C018F022C005
:1002800019F021C01AF020C01BF009C023F00AC0E9
:1002900022F00BC021F00CC020F0276A800E266EE1
:1002A000310E256E7E0E246ED2D918C027F019C0EB
:1002B00026F01AC025F01BC024F0D5D815BC03D0F9
:1002C0002A9C01D02A8A23501200186E14C027F0ED
:1002D00013C026F012C025F011C024F0B8D91BC0FD
:1002E00027F01AC026F019C025F018C024F0BBD0A2
:1002F00023C014F022C013F021C012F020C011F06E
:10030000170E276E720E266E310E256E7E0E246E2F
:1003100038D9EBD9096E0A90115006E012AE04D01C
:100320000A80096C800E121A106A0F6A0E6A7F0E1C
:1003300009240D6E170E276E720E266E310E256E75
:100340007E0E246E14C023F013C022F012C021F0E0
:1003500011C020F016D923C014F022C013F021C020
:1003600012F020C011F00950C8EC03F023C027F0B0
:1003700022C026F021C025F020C024F014C023F0B4
:1003800013C022F012C021F011C020F06AD823C09F
:1003900014F022C013F021C012F020C011F07D0E25
:1003A000236E880E226E590E216E720E206E14C0BE
:1003B00027F013C026F012C025F011C024F047D951
:1003C000E10E276E970E266E260E256E750E246E94
:1003D0004AD8C30E1B6E1D0E1A6E1E0E196E780EB5
:1003E00074DF5D0E1B6E500E1A6E630E196E7A0E60
:1003F0006CDF1B0E1B6EFE0E1A6E750E196E7C0ED8
:1004000064DF170E1B6E720E1A6E310E196E7E0EA1
:100410005CDF14C027F013C026F012C025F011C015
:1004200024F015D9276A266A256A7F0E246E1BD808
:1004300010C027F00FC026F00EC025F00DC024F02C
:1004400006D923C027F022C026F021C025F020C005
:1004500024F00AA01200236A226A216A7F0E206E0D
:1004600090D0800E251A2450205C296E11E2296C50
:10047000205024C020F0246E215025C021F0256E8C
:10048000225026C022F0266E235027C023F0276E6C
:100490001A0E296074D0245272E0286A21502C6E02
:1004A00025182B6E218E258E080E295E08E327C0A5
:1004B00028F026C027F025C026F0256AF5D7292682
:1004C00007E0D8902532263227322832292EF9D754
:1004D0002BAE33D02750235E2650225A2550215A66
:1004E00007E2D880000E235622562156800E2C1A81
:1004F000286C04E02306000E225A215A040E296EAD
:1005000021660DD022C021F023C022F028C023F0A4
:10051000286A080E205E29E3292EF2D726D021BEB4
:1005200008D0D8902836233622362136202EF7D709
:100530001CD028AE22D0286A0FD027502326265060
:1005400022222550212206E3213222322332283270
:10055000204A0DD028AE11D0233E0FD0223E0DD020
:10056000213E0BD0D8802390EFD7206A02D02A8278
:100570002068236A226A800E216E2CAE219E2350B1
:10058000120021501E6E25182B6E245051E020526F
:1005900052E0205E7F0E03E2202603E24BD02026AD
:1005A0004CE223C01CF022C01DF01E8E258E180EBA
:1005B0002C6E236A226A216A0BD027501C5C2650BD
:1005C0001D5811E31D6E1E6A27501C5E0BD004E2FD
:1005D00025501E5CF2E007E327501C5E26501D5A92
:1005E00025501E5AD8802336223621361C361D3619
:1005F0001E362C2EECD721BE07D020521BE02B320A
:1006000020062C2A2B36E3D707E227501C5E265003
:100610001D5A25501E5A17E3233E15D0223E13D0F3
:10062000213E11D0213222322332203E0CD005D07F
:100630002A8604D02A84206A02D02A822068236A6B
:10064000226A800E216E2BAE219E23501200215073
:100650001E6E25182B6E2050D8A424503AE0202678
:100660007E0E03E3205E03E336D0205E31E323C039
:100670001CF022C01DF01E8E258E236A226A216A7C
:10068000180E2C6E1E321D321C3206E32750232614
:1006900026502222255021222132223223322C2E92
:1006A000F1D721BE07D0233622362136205210E062
:1006B00020061E3416E3233E14D0223E12D0213EE3
:1006C00010D0D880213222322332203E0AD003D0EB
:1006D0002A84206A02D02A822068236A226A800E35
:1006E000216E2BAE219E2350120020C02CF02150F1
:1006F00023C021F0236E23362C3223322A6A23367C
:100700002C3602E32A842A7E06E12A802C6A236A98
:10071000226A216A0BD02C2803E0D880233206D02D
:10072000D890233202E12A8201D02A862AB604D048
:100730002AA20FD02AB407D07F0E236EFF0E226E9E
:10074000216E206E23D0800E236E01D0236A000E0E
:10075000F6D72AB0FBD7206A9F0E2C60EBD77E0E0F
:100760002C64F4D79E0E2C5C07E0D8902332223202
:10077000213220322C2AF6D72AA408D0D880000EA5
:10078000205621562256235623AEE0D72050120081
:10079000206E216A226A236A2B9E0AD02B9E23AEEA
:1007A00007D0D880000E20562156225623562B8E75
:1007B000960E2C6E235209E0080E2C2621C020F044
:1007C00022C021F023C022F011D022520FE1080EE6
:1007D0002C5E215007E1080E2C5E205002E12350D0
:1007E00010D0206A226E20C021F0206A22BE06D0DE
:1007F000D8902036213622362C06F8D72BAE229EF2
:100800002C5020C023F0206E225021C022F0216EF7
:100810001200400E2A6E006AB8964F0EAF6EB06A94
:10082000240EAC6E900EAB6E00010F0EC16E070E63
:10083000B46EC69AC30E926EE00E936EC00E946EA6
:100840009280928254D0F2A409D0F2942F4A302A96
:10085000D6CF2DF0D7CF2EF0817A11009EAA19D0D5
:10086000060EAB1412E1E2CF50F0E1CF4FF0512A67
:1008700010EE89F05150E126000EE222AECFE7FFE4
:1008800050C0E2FF4FC0E1FF1100AE50AE50AB9838
:10089000AB881100516A526A9D8A9F8AF28EF28C4F
:1008A00012009D9A00EE89F0010EF46EF36AF306D1
:1008B000000EF45AEE6AF450F310F9E1516A526AEC
:1008C0009D8A1200F29EE0CF0BF6D8CF0CF6E8CF4F
:1008D0000DF6F28E0001A192B36AB26AF29E0BC6C7
:1008E000E0FF0CC6D8FF0DC6E8FFF28E1000939A09
:1008F0008A8A0A0E12EC00F0939A8A9A9298899842
:1009000093948A94929489949296899693928A92D7
:1009100093968A9693988A98040ECA6ECB68BB6A9F
:100920000C0EBA6E9492040ECA6ECB68BE6A0C0EA0
:10093000BD6E9494CF0EBA16000EBA12000EBB6EA6
:10094000CF0EBD16000EBD12000EBE6E676A6B6A3A
:10095000400E6C6E706A6F6A6E6A7E0E6D6E746A9F
:10096000736A726A716E786A776A766A756A7C6A87
:100970007B6A7A6A796A94908B9094988B98949A0F
:100980008B9A94968B96B00E0EEC00F01E0E0EEC29
:1009900000F0000E0EEC00F04C6A416A4D9000EE43
:1009A00053F0140EEE68E82EFDD76880696A406A3D
:1009B00071DF77DFCD6AF294F28A870ED56EB16A65
:1009C000A192A082B36AB26AD08EA292B10EB16E29
:1009D000B1EC08F0B3EC0CF0B2EC0EF0050E6A6E60
:1009E000D6CF2DF0D7CF2EF017EC10F009C631F08E
:1009F000B10E315C06E3FE0E315C01E301D0336AD7
:100A0000E1D131AE37D0336A800E315C05E131C0BF
:100A100033F0346835682DD0900E315C05E131C07B
:100A200033F03668376825D0A00E315C05E131C05F
:100A300033F0386839681DD0B00E315C05E131C043
:100A400033F03A683B6815D0C00E315C04E131C028
:100A500033F03C680ED0D00E315C04E131C033F08D
:100A60003D6807D0E00E315C04E131C033F03E68F0
:100A70003F68A2D1335202E1A5D19ED1800E335CF2
:100A8000D8A451D0342803E131C034F04AD031C069
:100A900035F01D0E345C12E3590E345C0FE2800E0B
:100AA0000EEC00F034500EEC00F0000E0EEC00F0F6
:100AB000695201E06906346885D131D0780E345C22
:100AC00007E18B904190566855685468536827D069
:100AD000790E345C07E18B9841925A6859685868DE
:100AE00057681DD07A0E345C07E18B9A41945E689A
:100AF0005D685C685B6813D07B0E345C07E18B96A5
:100B000041966268616860685F6809D07C0E345CF9
:100B100004E1899A346856D102D0346853D13468DC
:100B20004C8050D149D1900E335CD8A42CD13628BA
:100B300003E131C036F026D131C037F04C80375256
:100B4000D8A444D01D0E365C11E3590E365C0EE27B
:100B5000800E0EEC00F036500EEC00F0000E0EECA5
:100B600000F0695201E069064C902FD0780E365C97
:100B700007E18B904190566855685468536825D0BA
:100B8000790E365C07E18B9841925A68596858682B
:100B900057681BD07A0E365C07E18B9A41945E68E9
:100BA0005D685C685B6811D07B0E365C07E18B96F4
:100BB00041966268616860685F6807D07C0E365C49
:100BC00003E1899A4C9001D04C90DBD040A0D9D061
:100BD0001D0E365C0FE3590E365C0CE2900E0EECE7
:100BE00000F036500EEC00F037500EEC00F0692AA1
:100BF0004C90C7D0780E365C2DE137C043F08B8027
:100C00007F0E435C21E2418002EE89F0D8904334AC
:100C1000E926000EEA22EECF07F0EFCF08F00750EA
:100C20002D24036E08502E20046E000E2F20056E1A
:100C3000000E3020066E03C053F004C054F005C00F
:100C400055F006C056F005D0419056685568546876
:100C5000536897D0790E365C2DE137C044F08B880D
:100C60007F0E445C21E2418202EE89F0D890443448
:100C7000E926000EEA22EECF07F0EFCF08F007508A
:100C80002D24036E08502E20046E000E2F20056EBA
:100C9000000E3020066E03C057F004C058F005C0A7
:100CA00059F006C05AF005D041925A685968586800
:100CB000576867D07A0E365C2DE137C045F08B8AD5
:100CC0007F0E455C21E2418402EE89F0D8904534E4
:100CD000E926000EEA22EECF07F0EFCF08F007502A
:100CE0002D24036E08502E20046E000E2F20056E5A
:100CF000000E3020066E03C05BF004C05CF005C03F
:100D00005DF006C05EF005D041945E685D685C6889
:100D10005B6837D07B0E365C2DE137C046F08B86A2
:100D20007F0E465C21E2418602EE89F0D89046347F
:100D3000E926000EEA22EECF07F0EFCF08F00750C9
:100D40002D24036E08502E20046E000E2F20056EF9
:100D5000000E3020066E03C05FF004C060F005C0D6
:100D600061F006C062F005D0419662686168606813
:100D70005F6807D07C0E365C03E1898A4C9001D015
:100D80004C90366819D0A00E335C0AE1382803E194
:100D900031C038F004D031C039F073EC10F00CD011
:100DA000B00E335C09E13A2803E131C03AF004D0D7
:100DB00031C03BF09CEC10F04CA004D037EC10F0AC
:100DC0000AC64BF0050E4B5CD8B02BD147502D5CBA
:100DD00048502E5849502F584A503058D8A013D157
:100DE0004A8E4B522AE141B006D08B905668556826
:100DF0005468536821D08270949002EE89F0D890A4
:100E00004334E926000EEA22EECF07F0EFCF08F0D8
:100E100007502D24036E08502E20046E000E2F2044
:100E2000056E000E3020066E03C053F004C054F06F
:100E300005C055F006C056F0E2D0010E4B5C2AE129
:100E400041B206D08B985A6859685868576821D0C3
:100E50008278949802EE89F0D8904434E926000E06
:100E6000EA22EECF07F0EFCF08F007502D24036EF3
:100E700008502E20046E000E2F20056E000E30202C
:100E8000066E03C057F004C058F005C059F006C004
:100E90005AF0B5D0020E4B5C2AE141B406D08B9AD1
:100EA0005E685D685C685B6821D0827A949A02EE25
:100EB00089F0D8904534E926000EEA22EECF07F0FB
:100EC000EFCF08F007502D24036E08502E20046E3B
:100ED000000E2F20056E000E3020066E03C05BF062
:100EE00004C05CF005C05DF006C05EF088D0030E63
:100EF0004B5C2AE141B606D08B96626861686068F7
:100F00005F6821D08276949602EE89F0D8904634BC
:100F1000E926000EEA22EECF07F0EFCF08F00750E7
:100F20002D24036E08502E20046E000E2F20056E17
:100F3000000E3020066E03C05FF004C060F005C0F4
:100F400061F006C062F05BD0040E4B5CD8A457D0B1
:100F50004DB00ED005EE09F0D8906B34E926000EA6
:100F6000EA22EECF7DF0EFCF7EF0806B7F6A0DD06E
:100F70007E6A7D6A05EE09F0D8906B34E926000E92
:100F8000EA22EECF7FF0EFCF80F04D7003EE89F0D4
:100F9000D8906734E926000EEA22EECF07F0EFCFB3
:100FA00008F007502D24036E08502E20046E000E0A
:100FB0002F20056E000E3020066E03C063F004C0C3
:100FC00064F005C065F006C066F000EE7DF0CF0E5F
:100FD000BD16EE38300BBD12ED30F36EEF30BE6E45
:100FE000F332BE3200EE7FF0CF0EBA16EE38300B81
:100FF000BA12ED30F36EEF30BB6EF332BB3237EC2A
:1010000010F00AC64BF030AE0BD0306A2F6A2E6A51
:101010002D6A416A00EE53F0140EEE68E82EFDD7FB
:1010200006D030AE04D0306A2F6A2E6A2D6AE86A84
:101030002EB6010F68B20108D8A490D0687268A0DB
:101040008DD0010E6A5C06E1695202E08B8601D008
:101050008B9684D0020E6A5C06E1695202E08B88AE
:1010600001D08B987BD0030E6A5C08E1695203E0E3
:101070008B888B8602D08B988B9670D0040E6A5C1E
:101080000DE1695208E068B203D08B988B8602D0DC
:101090008B888B9602D08B988B9660D0050E6A5CFD
:1010A0002DE169502AEC00F0326E325206E18B9647
:1010B0008B9A8B988B90899A20D0010E325C05E137
:1010C0008B868B9A8B988B9018D0020E325C05E140
:1010D0008B868B8A8B888B9010D0030E325C05E157
:1010E0008B868B8A8B888B8008D0040E325C05E15E
:1010F0008B868B8A8B888B80898A30D0060E6A5CBF
:1011000011E169B0828669A0829669B2828869A27B
:10111000829869B4828A69A4829A69B4828069A437
:1011200082901CD0070E6A5C11E169B0828869A0C8
:10113000829869B2828069A2829069B4828A69A425
:10114000829A69B4828669A4829608D0080E6A5C85
:1011500005E1695202E1899A01D0898A8170F0EF34
:1011600004F00201800E8A6F896B7D0E8C6F8B6B91
:10117000770E8E6F3D0E8D6F740E906F760E8F6FA3
:10118000710E926FBE0E916F6F0E946F180E936F6B
:101190006C0E966F810E956F690E986FF90E976FB2
:1011A000670E9A6F810E996F650E9C6F170E9B6F7D
:1011B000620E9E6FBC0E9D6F600EA06F6E0E9F6FD5
:1011C0005E0EA26F2F0EA16F5B0EA46FFD0EA36FBC
:1011D000590EA66FD80EA56F570EA86FC00EA76F39
:1011E000550EAA6FB40EA96F530EAC6FB40EAB6F51
:1011F000510EAE6FC10EAD6F4F0EB06FD90EAF6F07
:101200004D0EB26FFC0EB16F4C0EB46F2B0EB36F60
:101210004A0EB66F640EB56F480EB86FA80EB76F62
:10122000460EBA6FF70EB96F450EBC6F4F0EBB6F0F
:10123000430EBE6FB20EBD6F420EC06F1E0EBF6F6B
:10124000400EC26F930EC16F3F0EC46F120EC36F7C
:101250003D0EC66F990EC56F3C0EC86F2A0EC76F44
:101260003A0ECA6FC30EC96F390ECC6F640ECB6FC6
:10127000380ECE6F0D0ECD6F360ED06FBF0ECF6F06
:10128000350ED26F780ED16F340ED46F390ED36F06
:10129000330ED66F010ED56F310ED86FD10ED76FCA
:1012A000300EDA6FA80ED96F2F0EDC6F850EDB6F54
:1012B0002E0EDE6F6A0EDD6F2D0EE06F550EDF6FA6
:1012C0002C0EE26F460EE16F2B0EE46F3E0EE36FC5
:1012D0002A0EE66F3C0EE56F290EE86F400EE76FB1
:1012E000280EEA6F4A0EE96F270EEC6F590EEB6F6E
:1012F000260EEE6F6E0EED6F250EF06F890EEF6FFE
:10130000240EF26FA90EF16F230EF46FCE0EF36F61
:10131000220EF66FF80EF56F220EF86F280EF76F9B
:10132000210EFA6F5C0EF96F200EFC6F950EFB6FAD
:101330001F0EFE6FD20EFD6F03011F0E006F020124
:10134000140EFF6F03011E0E026F5B0E016F1D0E68
:10135000046FA60E036F1C0E066FF50E056F1C0EB4
:10136000086F480E076F1B0E0A6F9F0E096F1A0E4B
:101370000C6FFA0E0B6F1A0E0E6F590E0D6F190EC1
:10138000106FBC0E0F6F190E126F230E116F180E17
:10139000146F8D0E136F170E166FFA0E156F170E52
:1013A000186F6B0E176F160E1A6FDF0E196F160E71
:1013B0001C6F570E1B6F150E1E6FD10E1D6F150E75
:1013C000206F4F0E1F6F140E226FD00E216F140E60
:1013D000246F540E236F130E266FDA0E256F130E33
:1013E000286F640E276F120E2A6FF00E296F120EEF
:1013F0002C6F7F0E2B6F120E2E6F110E2D6F306F14
:10140000A50E2F6F110E326F3C0E316F100E346F20
:10141000D50E336F100E366F700E356F100E386F9D
:101420000E0E376F0F0E3A6FAE0E396F0F0E3C6F08
:10143000510E3B6F0E0E3E6FF50E3D6F0E0E406F60
:101440009C0E3F6F0E0E426F450E416F0D0E446FA6
:10145000F00E436F0D0E466F9D0E456F0D0E486FDB
:101460004B0E476F0C0E4A6FFC0E496F0C0E4C6F03
:10147000AF0E4B6F0C0E4E6F630E4D6F0C0E506F18
:10148000190E4F6F0B0E526FD10E516F0B0E546F22
:101490008A0E536F0B0E566F450E556F0B0E586F1D
:1014A000020E576F0A0E5A6FC00E596F0A0E5C6F0C
:1014B000800E5B6F0A0E5E6F410E5D6F0A0E606FED
:1014C000040E5F6F090E626FC80E616F090E646FC4
:1014D0008E0E636F090E666F550E656F090E686F8D
:1014E0001D0E676F080E6A6FE70E696F080E6C6F4E
:1014F000B20E6B6F080E6E6F7E0E6D6F080E706F02
:101500004B0E6F6F080E726F1A0E716F070E746FAD
:10151000E90E736F070E766FBA0E756F070E786F50
:101520008C0E776F070E7A6F5F0E796F070E7C6FE8
:10153000330E7B6F070E7E6F080E7D6F060E806F79
:10154000DE0E7F6F060E826FB50E816F060E846F02
:101550008D0E836F060E866F660E856F060E886F82
:10156000400E876F8A698969A20E8C6FC30E8B6FDC
:101570009A0E8E6F460E8D6F960E906F320E8F6F95
:10158000920E926F3A0E916F8E0E946F5D0E936F66
:101590008A0E966F9A0E956F860E986FF00E976F63
:1015A000830E9A6F5F0E996F7F0E9C6FE70E9B6F95
:1015B0007C0E9E6F850E9D6F790EA06F3B0E9F6F08
:1015C000760EA26F070EA16F720EA46FE80EA36FC6
:1015D0006F0EA66FDF0EA56F6C0EA86FEA0EA76FD9
:1015E0006A0EAA6F0A0EA96F670EAC6F3C0EAB6F46
:1015F000640EAE6F820EAD6F610EB06FDA0EAF6F1C
:101600005F0EB26F440EB16F5C0EB46FBF0EB36F5E
:101610005A0EB66F4C0EB56F570EB86FE90EB76F16
:10162000550EBA6F960EB96F530EBC6FBB6F510E4D
:10163000BE6F200EBD6F4E0EC06FFB0EBF6F4C0E07
:10164000C26FE50EC16F4A0EC46FDC0EC36F480E49
:10165000C66FE20EC56F460EC86FF50EC76F450E1A
:10166000CA6F150EC96F430ECC6F420ECB6F410E81
:10167000CE6F7B0ECD6F3F0ED06FC00ECF6F3E0E84
:10168000D26F100ED16F3C0ED46F6D0ED36F3A0E29
:10169000D66FD40ED56F390ED86F460ED76F370E72
:1016A000DA6FC20ED96F360EDC6F490EDB6F340E67
:1016B000DE6FDA0EDD6F330EE06F740EDF6F320E09
:1016C000E26F180EE16F300EE46FC50EE36F2F0E60
:1016D000E66F7B0EE56F2E0EE86F3A0EE76F2D0E6C
:1016E000EA6F020EE96F2B0EEC6FD10EEB6F2A0E34
:1016F000EE6FA90EED6F290EF06F880EEF6F280EBA
:10170000F26F6F0EF16F270EF46F5E0EF36F260E01
:10171000F66F530EF56F250EF86F500EF76F240E0F
:10172000FA6F540EF96F230EFC6F5E0EFB6F220EE4
:10173000FE6F6F0EFD6F0401210E006F0301860E18
:10174000FF6F0401200E026FA30E016F1F0E046FC6
:10175000C60E036F1E0E066FEF0E056F1E0E086F8E
:10176000076F1D0E0A6F520E096F1C0E0C6F8C0E48
:101770000B6F1B0E0E6FCB0E0D6F1B0E106F0F0E2F
:101780000F6F1A0E126F580E116F190E146FA50EEF
:10179000136F180E166FF80E156F180E186F4F0E88
:1017A000176F170E1A6FAB0E196F170E1C6F0A0EFC
:1017B0001B6F160E1E6F6F0E1D6F150E206FD70E4E
:1017C0001F6F150E226F430E216F140E246FB30E80
:1017D000236F140E266F270E256F130E286F9F0E92
:1017E000276F130E2A6F1A0E296F120E2C6F990E87
:1017F0002B6F120E2E6F1B0E2D6F110E306FA10E60
:101800002F6F110E326F290E316F100E346FB50E1F
:10181000336F100E366F440E356F0F0E386FD60EC5
:10182000376F0F0E3A6F6B0E396F0F0E3C6F030E52
:101830003B6F0E0E3E6F9D0E3D6F0E0E406F3A0ECB
:101840003F6F0D0E426FDA0E416F0D0E446F7C0E2E
:10185000436F0D0E466F210E456F0C0E486FC80E7C
:10186000476F0C0E4A6F720E496F0C0E4C6F1E0EB6
:101870004B6F0B0E4E6FCC0E4D6F0B0E506F7C0EE0
:101880004F6F0B0E526F2E0E516F0A0E546FE30EF8
:10189000536F0A0E566F990E556F0A0E586F510E00
:1018A000576F0A0E5A6F0B0E596F090E5C6FC80EF8
:1018B0005B6F090E5E6F850E5D6F090E606F450EE2
:1018C0005F6F090E626F060E616F080E646FC90EBE
:1018D000636F080E666F8E0E656F080E686F540E8C
:1018E000676F080E6A6F1C0E696F070E6C6FE50E4E
:1018F0006B6F070E6E6FAF0E6D6F070E706F7B0E06
:101900006F6F070E726F490E716F070E746F170EAF
:10191000736F060E766FE70E756F060E786FB90E51
:10192000776F060E7A6F8B0E796F060E7C6F5F0EE7
:101930007B6F060E7E6F340E7D6F060E806F0A0E73
:101940007F6F050E826FE10E816F050E846FB90EF9
:10195000836F050E866F930E856F050E886F6D0E73
:10196000876F000112000101040E8C6F880E8B6FCF
:10197000040E8E6FA60E8D6F040E906FB60E8F6FD5
:10198000040E926FC60E916F040E946FD60E936F75
:10199000040E966FE60E956F040E986FF60E976F15
:1019A000050E9A6F070E996F050E9C6F170E9B6FB1
:1019B000050E9E6F280E9D6F050EA06F390E9F6F4E
:1019C000050EA26F4B0EA16F050EA46F5D0EA36FE7
:1019D000050EA66F6E0EA56F050EA86F800EA76F81
:1019E000050EAA6F930EA96F050EAC6FA50EAB6F17
:1019F000050EAE6FB80EAD6F050EB06FCB0EAF6FAC
:101A0000050EB26FDF0EB16F050EB46FF20EB36F3D
:101A1000060EB66FB56FB86F1A0EB76F060EBA6FB7
:101A20002E0EB96F060EBC6F430EBB6F060EBE6F57
:101A3000580EBD6F060EC06F6D0EBF6F060EC26FE3
:101A4000830EC16F060EC46F980EC36F060EC66F6D
:101A5000AE0EC56F060EC86FC40EC76F060ECA6FF6
:101A6000DB0EC96F060ECC6FF20ECB6F070ECE6F7A
:101A7000090ECD6F070ED06F210ECF6F070ED26FFC
:101A8000380ED16F070ED46F500ED36F070ED66F7E
:101A9000690ED56F070ED86F810ED76F070EDA6FFC
:101AA0009A0ED96F070EDC6FB40EDB6F070EDE6F78
:101AB000CD0EDD6F070EE06FE70EDF6F080EE26FF1
:101AC000020EE16F080EE46F1D0EE36F080EE66F65
:101AD000380EE56F080EE86F530EE76F080EEA6FD9
:101AE0006F0EE96F080EEC6F8B0EEB6F080EEE6F4A
:101AF000A70EED6F080EF06FC40EEF6F080EF26FB9
:101B0000E10EF16F080EF46FF369090EF66F1D0E0A
:101B1000F56F090EF86F3B0EF76F090EFA6F5A0E4C
:101B2000F96F090EFC6F790EFB6F090EFE6F990EAF
:101B3000FD6F0201090E006F0101B90EFF6F020176
:101B4000090E026FD90E016F090E046FFA0E036FB2
:101B50000A0E066F1B0E056F0A0E086F3D0E076F0B
:101B60000A0E0A6F5F0E096F0A0E0C6F820E0B6F62
:101B70000A0E0E6FA50E0D6F0A0E106FC80E0F6FB6
:101B80000A0E126FEC0E116F0B0E146F110E136F05
:101B90000B0E166F360E156F0B0E186F5B0E176F50
:101BA0000B0E1A6F810E196F0B0E1C6FA70E1B6F99
:101BB0000B0E1E6FCE0E1D6F0B0E206FF50E1F6FDE
:101BC0000C0E226F1D0E216F0C0E246F460E236F1C
:101BD0000C0E266F6F0E256F0C0E286F980E276F58
:101BE0000C0E2A6FC20E296F0C0E2C6FED0E2B6F90
:101BF0000D0E2E6F180E2D6F0D0E306F430E2F6FC2
:101C00000D0E326F700E316F0D0E346F9C0E336FF0
:101C10000D0E366FCA0E356F0D0E386FF80E376F1A
:101C20000E0E3A6F260E396F0E0E3C6F550E3B6F3F
:101C30000E0E3E6F850E3D6F0E0E406FB60E3F6F5F
:101C40000E0E426FE70E416F0F0E446F180E436F7A
:101C50000F0E466F4B0E456F0F0E486F7E0E476F8F
:101C60000F0E4A6FB10E496F0F0E4C6FE60E4B6FA1
:101C7000100E4E6F1B0E4D6F100E506F500E4F6FAB
:101C8000100E526F870E516F100E546FBE0E536FB1
:101C9000100E566FF60E556F110E586F2E0E576FB1
:101CA000110E5A6F680E596F110E5C6FA20E5B6FAA
:101CB000110E5E6FDC0E5D6F120E606F180E5F6F9F
:101CC000120E626F540E616F120E646F910E636F8D
:101CD000120E666FCF0E656F130E686F0E0E676F74
:101CE000130E6A6F4D0E696F130E6C6F8E0E6B6F55
:101CF000130E6E6FCF0E6D6F140E706F110E6F6F2F
:101D0000140E726F540E716F140E746F980E736F01
:101D1000140E766FDC0E756F150E786F220E776FCE
:101D2000150E7A6F680E796F150E7C6FB00E7B6F93
:101D3000150E7E6FF80E7D6F160E806F410E7F6F51
:101D4000160E826F8C0E816F160E846FD70E836F06
:101D5000170E866F230E856F170E886F700E876FB4
:101D6000000112000401896B170E8A6F200E8B6F21
:101D7000270E8C6F2D0E8D6F330E8E6F370E8F6F7B
:101D80003C0E906F400E916F440E926F480E936F11
:101D90004B0E946F4E0E956F520E966F550E976FB9
:101DA000580E986F5B0E996F5D0E9A6F600E9B6F69
:101DB000630E9C6F650E9D6F680E9E6F6A0E9F6F1F
:101DC0006D0EA06F6F0EA16F710EA26F730EA36FD9
:101DD000760EA46F780EA56F7A0EA66F7C0EA76F95
:101DE0007E0EA86F800EA96F820EAA6F840EAB6F55
:101DF000860EAC6F880EAD6F8A0EAE6F8B0EAF6F16
:101E00008D0EB06F8F0EB16F910EB26F930EB36FD8
:101E1000940EB46F960EB56F980EB66F990EB76F9D
:101E20009B0EB86F9D0EB96F9E0EBA6FA00EBB6F62
:101E3000A20EBC6FA30EBD6FA50EBE6FA60EBF6F28
:101E4000A80EC06FA90EC16FAB0EC26FAC0EC36FF0
:101E5000AE0EC46FAF0EC56FB10EC66FB20EC76FB8
:101E6000B40EC86FB50EC96FB60ECA6FB80ECB6F81
:101E7000B90ECC6FBB0ECD6FBC0ECE6FBD0ECF6F4B
:101E8000BF0ED06FC00ED16FC10ED26FC30ED36F15
:101E9000C40ED46FC50ED56FC70ED66FC80ED76FE0
:101EA000C90ED86FCA0ED96FCC0EDA6FCD0EDB6FAC
:101EB000CE0EDC6FCF0EDD6FD10EDE6FD20EDF6F78
:101EC000D30EE06FD40EE16FD50EE26FD70EE36F45
:101ED000D80EE46FD90EE56FDA0EE66FDB0EE76F12
:101EE000DD0EE86FDE0EE96FDF0EEA6FE00EEB6FDE
:101EF000E10EEC6FE20EED6FE30EEE6FE50EEF6FAD
:101F0000E60EF06FE70EF16FE80EF26FE90EF36F79
:101F1000EA0EF46FEB0EF56FEC0EF66FED0EF76F49
:101F2000EE0EF86FEF0EF96FF10EFA6FF20EFB6F17
:101F3000F30EFC6FF40EFD6FF50EFE6FF60EFF6FE5
:101F40000501F70E006FF80E016FF90E026FFA0E21
:101F5000036FFB0E046FFC0E056FFD0E066FFE0E89
:101F6000076F08690001326A800E325CD8B05DD01C
:101F7000330E276E266E4B0E256E820E246E325067
:101F8000C8EC03F0C1EC02F020C081F021C082F067
:101F900022C083F023C084F0066A056A046A800EBA
:101FA000036E10EE03F081C011F082C012F083C006
:101FB00013F084C014F033EC00F020C085F021C091
:101FC00086F022C087F023C088F085C020F086C04C
:101FD00021F087C022F088C023F075EC03F005EEF5
:101FE00009F0D8903234E926000EEA2220C0EEFF34
:101FF00021C0EFFF05EE09F0D8903234E926000E3B
:10200000EA22EECF03F0EFCF04F0040E045C0AE303
:1020100005EE09F0D8903234E926000EEA22EE6887
:10202000030EEF6E322AD8A09FD71200FFD751506F
:10203000525C16E0522AEACF0AF0E9CF09F000EE2E
:1020400089F05250E926000EEA22EF500601096F8E
:102050000AC0EAFF09C0E9FFD8801200000105D0DC
:10206000E8680601096FD8A01200000112000601FD
:102070000A694A8E326A0001D8903234E96EEA6AFF
:10208000EA36E936EA36530EE926000EEA22EFCFA9
:1020900003F0ECCF04F0ECCF05F0ECCF06F04750A6
:1020A000035C48500458495005584A50065815E2F8
:1020B000D8903234E96EEA6AEA36E936EA36530EE7
:1020C000E926000EEA22EFCF47F0ECCF48F0ECCF44
:1020D00049F0ECCF4AF032C00AF6322A050E325CE3
:1020E000CAE34C9012001D0E385C0DE3590E385CAB
:1020F0000AE2A00E0EEC00F038500EEC00F0395061
:102100000EEC00F017D0780E385C03E139C043F0D4
:1021100011D0790E385C03E139C044F00BD07A0E4F
:10212000385C03E139C045F005D07B0E385C02E134
:1021300039C046F038681200060E3A5CD8A4BAD00E
:102140003BC067F0675236E005EE09F0D8906B347B
:10215000E926000EEA22EECF7DF0EFCF7EF005EE0D
:1021600009F0D8906B34E926000EEA22EECF7FF01A
:10217000EFCF80F003EE89F0D8906734E926000EA7
:10218000EA22EECF07F0EFCF08F007502D24036EC0
:1021900008502E20046E000E2F20056E000E3020F9
:1021A000066E03C063F004C064F005C065F006C0AD
:1021B00066F064D005EE09F0D8906B34E926000E85
:1021C000EA22EECF03F0EFCF04F003C020F004C00A
:1021D00021F0CAEC03F06DC024F06EC025F06FC092
:1021E00026F070C027F027EC03F020C075F021C066
:1021F00076F022C077F023C078F005EE09F0D89091
:102200006B34E926000EEA22EECF03F0EFCF04F0A4
:1022100003C020F004C021F0CAEC03F071C024F028
:1022200072C025F073C026F074C027F027EC03F0CD
:1022300020C079F021C07AF022C07BF023C07CF06E
:1022400075C020F076C021F077C022F078C023F06E
:1022500075EC03F07D6E21C07EF079C020F07AC06D
:1022600021F07BC022F07CC023F075EC03F07F6E80
:1022700021C080F0666865686468636800EE7DF080
:10228000CF0EBD16EE38300BBD12ED30F36EEF30D1
:10229000BE6EF332BE3200EE7FF0CF0EBA16EE38CD
:1022A000300BBA12ED30F36EEF30BB6EF332BB324F
:1022B0004C809DD1070E3A5CD8A47DD03BC06BF01A
:1022C00005EE09F0D8903B34E926000EEA22EECF65
:1022D00003F0EFCF04F003C020F004C021F0CAECFB
:1022E00003F06DC024F06EC025F06FC026F070C002
:1022F00027F027EC03F020C075F021C076F022C053
:1023000077F023C078F005EE09F0D8903B34E92649
:10231000000EEA22EECF03F0EFCF04F003C020F06E
:1023200004C021F0CAEC03F071C024F072C025F0A3
:1023300073C026F074C027F027EC03F020C079F0BA
:1023400021C07AF022C07BF023C07CF075C020F061
:1023500076C021F077C022F078C023F075EC03F04E
:102360007D6E21C07EF079C020F07AC021F07BC064
:1023700022F07CC023F075EC03F07F6E21C080F06A
:1023800000EE7DF0CF0EBD16EE38300BBD12ED30F5
:10239000F36EEF30BE6EF332BE3200EE7FF0CF0E42
:1023A000BA16EE38300BBA12ED30F36EEF30BB6E6A
:1023B000F332BB321CD10A0E3A5CD8A4A7D03BC082
:1023C0006CF0276A266A7E0E256E850E246E6C5090
:1023D000C8EC03F0C1EC02F020C06DF021C06EF03B
:1023E00022C06FF023C070F06DC024F06EC025F0E5
:1023F0006FC026F070C027F0236A226A216A7F0E20
:10240000206E31EC02F020C071F021C072F022C0C9
:1024100073F023C074F005EE09F0D8906B34E92610
:10242000000EEA22EECF03F0EFCF04F003C020F05D
:1024300004C021F0CAEC03F06DC024F06EC025F09A
:102440006FC026F070C027F027EC03F020C075F0B5
:1024500021C076F022C077F023C078F005EE09F0B5
:10246000D8906B34E926000EEA22EECF03F0EFCFCE
:1024700004F003C020F004C021F0CAEC03F071C0E6
:1024800024F072C025F073C026F074C027F027EC4A
:1024900003F020C079F021C07AF022C07BF023C085
:1024A0007CF075C020F076C021F077C022F078C0B3
:1024B00023F075EC03F07D6E21C07EF079C020F032
:1024C0007AC021F07BC022F07CC023F075EC03F0D1
:1024D0007F6E21C080F000EE7DF0CF0EBD16EE388D
:1024E000300BBD12ED30F36EEF30BE6EF332BE3204
:1024F00000EE7FF0CF0EBA16EE38300BBA12ED3088
:10250000F36EEF30BB6EF332BB3271D01E0E3A5C0D
:1025100012E13BC043F03BC044F03BC045F03BC040
:1025200046F0B00E0EEC00F01E0E0EEC00F03B502C
:102530000EEC00F05CD0420E3A5C19E13B5202E135
:1025400058D801D065D868D8B00E0EEC00F0420E15
:102550000EEC00F03B500EEC00F0B00E0EEC00F074
:102560001E0E0EEC00F0000E0EEC00F040D0450EFA
:102570003A5C23E13B5202E0688001D06890696ACE
:102580008B908B988B9A8B96899A5668556854686D
:1025900053685A685968586857685E685D685C682F
:1025A0005B686268616860685F683BC06AF0090EDA
:1025B0006A5C02E3080E6A6E1AD07B0E3A5C17E181
:1025C000416A8B908B988B9A899A8B96696A00EEF8
:1025D00053F0140EEE68E82EFDD74C80B00E0EECD2
:1025E00000F07B0E0EEC00F0000E0EEC00F03A68EE
:1025F000120089988A94416A436A446A456A466A25
:102600008B908B988B9A8B96899A696A409012006E
:1026100089888A84408012006B6A676A400E6C6EFB
:10262000CF0EBD16000EBD12000EBE6ECF0EBA1636
:10263000000EBA12000EBB6E050E6A6E00EE53F06D
:10264000140EEE68E82EFDD74C80706A6F6A6E6AD1
:102650007E0E6D6E746A736A726A716E68801200A3
:020000040030CA
:0300010006160ED2
:020005008580F4
:060008000FC00FE00F40E5
:00000001FF
